:100000000C94E5000C94F80F0C94D10F0C94AA0FEB
:100010000C94830F0C940D010C940D010C945C0F47
:100020000C940D010C944D120C94DF170C94511884
:100030000C940D010C940D010C940D010C940D0108
:100040000C940D010C940D010C940D010C940D01F8
:100050000C940D010C940D010C940D010C94120FD5
:100060000C940D010C94BC1A0C94961A0C940D016E
:100070000C940D010C940D010C940D010C940D01C8
:100080000C940D010C940D010C940D010C940D01B8
:100090000C9406050C940D010C940D010C940D01AB
:1000A0000C940D010C940A030C940D010F0C120C0E
:1000B000010C050C0B0C330C330C330C160C1A0C06
:1000C0001E0C240C280C330C2E0C00000000240005
:1000D00027002A002D003000000000002500280025
:1000E0002B002E0031000000000023002600290014
:1000F0002C002F000404040404030405020202027D
:1001000004030202020206060606060604040202B0
:100110000204040408020110408040102040804086
:10012000800802040180402010020110801020404D
:1001300040200000000200090F0000030401000C31
:1001400000000000000000000000000000000000AF
:1001500000080B0002020201000904000001020273
:1001600000000524001001052401010104240206F9
:100170000524060001070581031000400904010061
:10018000020A000000070502024000000705830282
:100190004000000403090412010002EF0201404183
:1001A00023368000010102030141726475696E6F9C
:1001B000204C4C430041726475696E6F204C656F32
:1001C0006E6172646F00E423211D11241FBECFEF06
:1001D000DAE0DEBFCDBF12E0A0E0B1E0E2EAF4E594
:1001E00002C005900D92A031B107D9F724E0A0E13B
:1001F000B2E001C01D92A73EB207E1F710E0C4EEE5
:10020000D0E004C02197FE010E942C27C33ED107F5
:10021000C9F70E94501D0C94442A0C9400002F92A0
:100220003F924F925F926F927F928F929F92AF9286
:10023000BF92CF92DF92EF92FF920F931F93CF93D3
:10024000DF93CDB7DEB727970FB6F894DEBF0FBEAA
:10025000CDBF9F838E831B014D83809165028111E9
:100260001BC081E080936502109272001092C00062
:1002700094E09093C10099E09093C2008093C300F2
:1002800083E08093BF0088EE8093D1001092BF007E
:100290001092D200579A7894109209012E813F81D2
:1002A00037FF05C03F773F832E830AE001C001E09E
:1002B00088E2089F802D112490E04E815F814817CD
:1002C000590708F4C2C0013039F44131574220F0D7
:1002D000E0E1F7E2FF83EE83802E912CA12CB12C7C
:1002E0008E819F81969587959C0140E050E02983FF
:1002F0003A834B835C834E815F812A01612C712C90
:10030000A501940160E072E18AE790E00E94E8268E
:1003100029813A814B815C81620F731F841F951F75
:10032000A30192010E94A62569017A01EE24FF240F
:1003300010E01F5FC11434E0D306E104F10408F1BA
:1003400020E032E14AE750E0012E04C05595479580
:10035000379527950A94D2F7C501B4010E94E82683
:1003600029813A814B815C81620F731F841F951F25
:10037000A30192010E94A62569017A01EE24FF24BF
:10038000D8CF0A3049F48E819F8105966AE070E0EB
:100390000E9404277F836E834E815F81483E83E005
:1003A000580759F09101DA010E94312628EE33E016
:1003B00040E050E00E94A625190110927200809141
:1003C000C100807F182B1093C100BB27AF2D9E2D3D
:1003D0008D2D8093BF00C092D1002D81203108F077
:1003E0002FE080E190E0821B910904C0F694E7942D
:1003F000D794C7948A95D2F78D2D99278093BF0003
:10040000C092D200309267022092660289B38FEFC9
:1004100089BB84E08093720027960FB6F894DEBF04
:100420000FBECDBFDF91CF911F910F91FF90EF9045
:10043000DF90CF90BF90AF909F908F907F906F9004
:100440005F904F903F902F9008959F838E8344CF6D
:1004500085ED8093BC008091BC0084FDFCCF1092A0
:10046000F102089540913D02262F30E0240F311D06
:1004700021323105DCF42091F1022430C9F4FC0171
:1004800080E090E0861758F430913D022191DC0124
:10049000A55EBD4FA30FB11D2C930196F3CF8091A4
:1004A0003D02680F60933D0280E0089581E0089569
:1004B00082E008950895E091AA028091A902E817C8
:1004C00030F4F0E0E555FD4F808190E008958FEF26
:1004D0009FEF08959091AA028091A902981750F475
:1004E000E92FF0E0E555FD4F208130E09F5F9093CC
:1004F000AA0202C02FEF3FEFC90108958091A9021F
:1005000090E02091AA02821B91090895CF92DF9278
:10051000EF92FF920F931F93CF93DF937C01262FCF
:10052000972F8A018091F202882391F0C62FD72F4E
:100530006E01C40ED51ECC15DD0571F06991D70191
:10054000ED91FC910190F081E02DC7010995F3CF69
:10055000642F822F0E943202C801DF91CF911F9138
:100560000F91FF90EF90DF90CF900895CF93DF939E
:100570001F92CDB7DEB769832091F2022223D1F01A
:1005800020911403203240F021E030E0FC0133835D
:10059000228380E090E015C08091F302E82FF0E024
:1005A000EC50FD4F998190838F5F8093F30280938D
:1005B000140305C061E0CE0101960E94320281E081
:1005C00090E00F90DF91CF910895089580E090E042
:1005D000089580916802E0916902F0916A0288238F
:1005E00011F0849101C080819FEB980F9A3110F433
:1005F000805E0895803269F42091690230916A0228
:10060000A9014F5F5F4F50936A0240936902232B09
:1006100001F708951F920F920FB60F9211246F9257
:100620007F928F929F92AF92BF92CF92DF92EF9282
:10063000FF920F931F932F933F934F935F936F936B
:100640007F938F939F93AF93BF93CF93DF93EF935A
:10065000FF9380916602909167029C0121503109BD
:100660003093670220936602892B09F0B0C1109283
:10067000720078948091C100807F84608093C10073
:1006800083E08093BF0088EE8093D1001092BF007A
:100690001092D20081E080930901809169029091CB
:1006A0006A02892B09F493C18091640281118FC180
:1006B0009090080180916302882321F0809162026A
:1006C00081117BC17724739470ECA72E7DE5B72E42
:1006D000EAE06E2EF4E08F2EA0EDCA2EA7E0DA2E0F
:1006E000B4E0EB2EF12C04EF11E0CFE0D0E00E945B
:1006F000E9022091690230916A022F5F3F4F3093E7
:100700006A0220936902853609F45EC07CF5813661
:1007100009F49EC024F58C3309F452C08E3309F4D9
:100720004DC0813209F08FC080920801D09205013E
:10073000C0920401F0920701E092060110930301B8
:1007400000930201D0930101C09300011092630253
:10075000909008018091020190910301C8CF8336E7
:1007600089F10CF478C000E022E077C08D36A9F161
:100770006CF4873679F15CF18C3609F064C00E9424
:100780009E1290930701809306014EC08237D1F1EB
:100790004CF48F3609F057C00E949E12982E809319
:1007A0000801A5CF843789F1863709F04CC00E9433
:1007B0009E12909301018093000199CF939497CF5B
:1007C0009A9495CF00E01FC000E024E046C000E00E
:1007D00025E043C000E027E040C00E94E9028C36DB
:1007E00019F41092630204C07092630210926202C4
:1007F0008091690290916A02019690936A028093B7
:10080000690275CF01E020E028C00E949E12BC0161
:10081000C5010E940427669EC001679E900D1124A9
:10082000909305018093040180910401909105014A
:1008300060910601709107010E94042770930301E3
:100840006093020154CF10926A0210926902BFC0F5
:1008500000E029E002C000E02BE0122F3CE0939E74
:10086000100D11240E94E902982F977F933259F4BA
:100870008091690290916A02019690936A02809336
:1008800069021F5FEFCF8D3269F480916902909108
:100890006A02019690936A028093690211500E9445
:1008A000E902F1CFC0910201D09103018153883058
:1008B00058F4C0910401D09105010E949E12BC0120
:1008C000CE010E940427EB017E01F694E7940E947A
:1008D000E9028E3261F48091690290916A02019678
:1008E00090936A0280936902CE0DDF1DEECFFE0168
:1008F00080916302882349F0CE0196958795809375
:10090000620280916202E81BF109C0910001D0915E
:100910000101011104C01F3F11F0C11105C040E0E9
:10092000BF0188EE93E046C0113130F020EF210F77
:10093000203618F02FE501C020E0822F6CE00E94E5
:10094000F826682F74EF7603A0011124BA01620F14
:10095000711D9B016C30710540F4220F331FD901CA
:10096000A65CBE4F2D913C9102C020E030E0873064
:1009700081F0082E02C0220F331F0A94E2F7823062
:1009800028F0C90105966AE070E00CC0C9019058D2
:100990000CC0C90126E0880F991F2A95E1F702963D
:1009A00065E070E00E940427CB014C2FC03108F0B5
:1009B0004FE0BF010E940F010AC06091620270E027
:1009C00040E088EE93E00E940F0110926202FF91D6
:1009D000EF91DF91CF91BF91AF919F918F917F91D7
:1009E0006F915F914F913F912F911F910F91FF90C8
:1009F000EF90DF90CF90BF90AF909F908F907F90BF
:100A00006F900F900FBE0F901F9018951F920F922E
:100A10000FB60F9211242F933F934F935F936F93D1
:100A20007F938F939F93AF93BF93EF93FF938091A7
:100A3000B900887F803609F49CC068F5883209F4D3
:100A40005BC090F4803109F454C038F4882309F471
:100A5000F6C0883009F44DC0F6C0883109F44CC0A6
:100A6000803209F45DC0EFC0803409F468C048F4F6
:100A7000803309F455C0883309F0E5C08093EF0254
:100A8000D8C0803509F44FC0883509F45DC088347A
:100A900009F0D9C0D6C0883909F4C7C0A8F488378E
:100AA00009F467C038F4883609F463C0803709F464
:100AB00060C0C9C0883809F4B8C0803909F45FC083
:100AC000803809F0C0C05BC0803B09F486C038F4B0
:100AD000803A09F466C0883A09F47FC0B4C0803C0B
:100AE00009F4A7C0883C09F4A4C0883B09F48AC073
:100AF000AAC08091CC0210C09091EE028091ED02CC
:100B0000981770F5E091EE0281E08E0F8093EE026F
:100B1000F0E0E353FD4F80818093BB0085EC86C0FD
:100B20008093EF028EC0E091EE0281E08E0F809301
:100B3000EE028091BB00F0E0E353FD4F8083909183
:100B4000EE028091ED026EC0E091EE0281E08E0F28
:100B50008093EE028091BB00F0E0E353FD4F808371
:100B60008091F00281116DC081E08093CB0284EA14
:100B700061C083E08093F10210926102CFCF809137
:100B80006102803208F051C0E091610281E08E0F75
:100B9000809361028091BB00F0E0EF5BFD4F8083AA
:100BA000BDCF85EC8093BC001092F1028091610270
:100BB000803230F4E0916102F0E0EF5BFD4F108293
:100BC0006091610270E0E0913F02F091400281E4A7
:100BD00092E009951092610236C084E08093F102A0
:100BE00010923E0210923D02E0913B02F0913C02D5
:100BF000099580913D02811105C081E080933D02FD
:100C000010921B02E0913E0281E08E0F80933E0223
:100C1000F0E0E55EFD4F80818093BB0090913E0245
:100C200080913D02981708F479CF85E88093BC0045
:100C30000AC085EC8093BC001092F10204C01092AF
:100C4000EF020E942802FF91EF91BF91AF919F9117
:100C50008F917F916F915F914F913F912F910F9065
:100C60000FBE0F901F90189580911202811105C040
:100C700081E0809312020E940812F89480916D0224
:100C800090916E02789490931402809313026EE810
:100C900073E00E94182770931802609317028091E6
:100CA0001202811105C081E0809312020E94081295
:100CB000F89480916B0290916C0278949093160254
:100CC000809315026EE873E00E94182770931A0251
:100CD0006093190208958F929F92AF92BF92CF9224
:100CE000DF92EF92FF920F931F930E94B013E09058
:100CF0006D04F0906E0480918A0290918B02E81A44
:100D0000F90AF0921102E09210020E94880D2091DF
:100D1000880230918902AB01421B530B9A017093F8
:100D2000890260938802D7010E94322720E030E0D8
:100D300040EE50E00E943927EDE8AE2EF8E3BF2EDA
:100D4000ACE0CA2EDD24D394E12CF12C00E010E0BD
:100D50000E94752749015A01809190029091910259
:100D6000A0919202B0919302880D991DAA1DBB1DFE
:100D70008093900290939102A0939202B093930279
:100D80009D01552737FD5095452FA8E6B1E00E94FB
:100D9000C525BB2797FDB095AB2F80938C02909310
:100DA0008D02A0938E02B0938F021F910F91FF903E
:100DB000EF90DF90CF90BF90AF909F908F9008956D
:100DC000EF92FF920F931F93CF93DF93CDB7DEB7D0
:100DD00028970FB6F894DEBF0FBECDBF61E0CE01FD
:100DE00001960E94E01B82E8E82E82E0F82E8981BD
:100DF0009A81F70120813181821B930B98878F8321
:100E0000BE01695F7F4F8CE594E00E941F1008E9E6
:100E100012E0F801918380838B819C81F70122810C
:100E20003381821B930B98878F83BE01695F7F4F4D
:100E30008FE494E00E941F10F801938382838D81D8
:100E40009E81F70124813581821B930B98878F83C4
:100E5000BE01695F7F4F82E494E00E941F10F80199
:100E60009583848328960FB6F894DEBF0FBECDBF5E
:100E7000DF91CF911F910F91FF90EF900895CF9246
:100E8000DF92EF92FF920F931F93CF93DF93CDB733
:100E9000DEB72C970FB6F894DEBF0FBECDBF10E0C3
:100EA0008091C404181788F4E091C204F091C3043F
:100EB00083E0189FE00DF11D112480818F3118F41B
:100EC00062E00E941E0D1F5FEBCF8091C5048F3141
:100ED00070F460E00E94EE0C61E08091C5040E9415
:100EE0001E0D8091CD049091CE040E947D0D8091C5
:100EF000C6049091C704892B01F58CE0EEE2F1E085
:100F0000DE01119601900D928A95E1F76CE070E098
:100F100080E090E00E946529009779F02CE0FE01C6
:100F20003196DC0101900D922A95E1F79093C70468
:100F30008093C60486E08093C8042091C204309157
:100F4000C30480E09091C404891750F4F90193E040
:100F5000899FE00DF11D1124128211828F5FF2CF63
:100F600010E08091C804181708F07EC09091C60464
:100F70008091C704E92FF82FE10FF11DE10FF11D5A
:100F8000C080D1804091C9045091CA04B60180E06C
:100F900090E00E94DB118091CB049091CC040E94E0
:100FA0007D0D00E08091C4040817E0F483E0089F01
:100FB00070011124E091C204F091C304EE0DFF1DF5
:100FC00080818F3168F40E94C50C892B49F4E0912F
:100FD000C204F091C304EE0DFF1D81818F5F8183F8
:100FE0000F5FE0CF0E94C1118091CD049091CE049B
:100FF0000E947D0D4091C9045091CA04B60181E060
:1010000090E00E94DB118091CB049091CC040E946F
:101010007D0D00E08091C4040817E0F493E0099F7F
:1010200070011124E091C204F091C304EE0DFF1D84
:1010300080818F3168F40E94C50C892B49F4E091BE
:10104000C204F091C304EE0DFF1D82818F5F828385
:101050000F5FE0CF0E94C1118091CD049091CE042A
:101060000E947D0D1F5F7DCF84E10E94C812909188
:10107000C404891758F4E091C204F091C30493E0CA
:10108000899FE00DF11D1124818101C080E090E075
:101090009A838983BE016F5F7F4F85E394E00E944E
:1010A0001F1080939E0286E10E94C8129091C40492
:1010B000891758F4E091C204F091C30493E0899F2A
:1010C000E00DF11D1124818101C080E090E09A8340
:1010D0008983BE016F5F7F4F88E294E00E941F10FA
:1010E00080939F0286E10E94C8129091C4048917E0
:1010F00058F4E091C204F091C30493E0899FE00D9D
:10110000F11D1124828101C080E090E09A838983DF
:10111000BE016F5F7F4F8BE194E00E941F108093B0
:10112000A00284E00E94C8129091C404891758F468
:10113000E091C204F091C30493E0899FE00DF11D9A
:101140001124828101C080E090E09A838983BE01EE
:101150006F5F7F4F8EE094E00E941F108093A1028A
:101160002C960FB6F894DEBF0FBECDBFDF91CF91A6
:101170001F910F91FF90EF90DF90CF9008950E9404
:10118000060F2091960230919702621B730B7093A9
:101190009502609394020895882311F0479A01C044
:1011A00047983F9A08954F925F926F927F928F92E5
:1011B0009F92AF92BF92CF92DF92EF92FF92CF9326
:1011C000DF930E94060F4B015C017B010E94060F1A
:1011D000EB01C819D9098091980290919902875919
:1011E00091098D359140C8F581E00E94CC0880902E
:1011F000140190901501A0901601B0901701A5015F
:10120000940160E070E088EC91E40E9440260E9426
:10121000B2262B013C01A501940160E070E080ED55
:1012200092E40E9440260E94B226DC01CB01B2016A
:101230000E947411C436D10508F084C00E94060FC4
:10124000EB01CE19DF090E94E00680919C0290918B
:101250009D028937910574F375C080919C0290912D
:101260009D02895791098B379140C8F581E00E9412
:10127000CC088090140190901501A0901601B090B8
:101280001701A501940160E070E088EC92E40E94EF
:1012900040260E94B2262B013C01A501940160E08A
:1012A00070E080ED91E40E9440260E94B226DC01AD
:1012B000CB01B2010E947411C436D10508F042C0BE
:1012C0000E94060FEB01CE19DF090E94E006809113
:1012D0009802909199028739910574F333C05D9813
:1012E000559AC0901401D0901501E0901601F0902D
:1012F0001701A701960160E070E088EC92E40E947B
:1013000040260E94B2264B015C01A701960160E0D5
:1013100070E080ED92E40E9440260E94B226DC013B
:10132000CB01B401DF91CF91FF90EF90DF90CF9090
:10133000BF90AF909F908F907F906F905F904F90F5
:101340000C947411DF91CF91FF90EF90DF90CF90CC
:10135000BF90AF909F908F907F906F905F904F90D5
:10136000089581E00E94CC0881E090E00E94531C27
:101370000E94E0068091980290919902855F9140C9
:101380008B34944050F420919A0230919B022D525C
:10139000314081E0233F314008F080E020919C0201
:1013A00030919D02255F31402B34344008F02AC132
:1013B00020919A0230919B022D523140233F3140BF
:1013C00008F020C1882309F495C00E94472522E037
:1013D00030E040E050E00E94A625DC01CB01019600
:1013E000A11DB11D81309105A105B10509F0B6C15E
:1013F0006EE670E088E690E00E9474110E94060F8D
:1014000070939702609396020E94BF0880919402A5
:1014100090919502883E934048F40E94BF086EE682
:1014200070E088E690E00E947411F0CF0E94E00620
:1014300080919802909199028639910584F4809167
:101440009C0290919D02883791054CF40E94E00621
:1014500064E670E088E690E00E947411E9CF109293
:1014600090021092910210929202109293021092A6
:101470008C0210928D0210928E0210928F020E94A6
:101480006B0680918C0290918D02A0918E02B0919A
:101490008F028A359105A105B1052CF50E946B06D6
:1014A0000E94E00680919C0290919D0289579109CB
:1014B0008B37914028F464E670E080E090E010C043
:1014C00080919802909199028759910964E670E0A1
:1014D0008D35914018F484E390E002C08AE190E0F9
:1014E0000E947411CECF64E670E088E690E00E941E
:1014F000741165C00E94472522E030E040E050E0D2
:101500000E94A625613009F07FC0109290021092CF
:101510009102109292021092930210928C021092F9
:101520008D0210928E0210928F0210921802109269
:1015300017020E946B0680918C0290918D02A091FF
:101540008E02B0918F02893D9F4FAF4FBF4FACF0DD
:101550000E946B060E9434060E94E00669E170E07A
:1015600088E690E00E94741180919802909199020F
:10157000875991098D359140F0F60E946B060E94C3
:10158000060F709397026093960280918C0290915F
:101590008D02A0918E02B0918F028C3A9F4FAF4F77
:1015A000BF4F6CF00E94BF080E946B060E94E006CD
:1015B0008091940290919502893B9B4020F080E0BD
:1015C00090E00C94531C8091980290919902875955
:1015D00091098D35914018F460E070E00EC0809163
:1015E0009C0290919D02895791098B37914018F484
:1015F00062E370E002C069E170E088E690E00E947A
:101600007411C3CF81111CC064E670E088E690E0DD
:101610000E9474110E94060F7093970260939602C5
:101620000E94BF088091940290919502883E934059
:1016300030F60E94BF080E94E0060E94D308F2CF55
:101640000E94472522E030E040E050E00E94A625BD
:101650006130D1F610929002109291021092920293
:101660001092930210928C0210928D0210928E02B0
:1016700010928F0210921A02109219020E946B06A9
:1016800080918C0290918D02A0918E02B0918F0278
:101690008897A105B1055CF40E946B060E94340690
:1016A00064E670E08AE190E00E947411E9CF109244
:1016B0001A02109219020E946B0680918C0290917E
:1016C0008D02A0918E02B0918F0285359105A10502
:1016D000B1055CF40E946B060E94340664E670E07B
:1016E0008AE190E00E947411E8CF64E670E088E639
:1016F00090E00E9474110E94060F7093970260930D
:1017000096020E94BF088091940290919502883EB3
:10171000934068F40E94BF080E94E00680919C02FA
:1017200090919D02895791098B37914060F70E94F3
:10173000060F70939702609396020E94BF088091F3
:10174000940290919502883E934008F038CF0E9411
:10175000BF080E94E0060E94D308F1CF823009F44E
:10176000D4CE52CF80E090E0892B29F00E94191747
:1017700081110C9400000895CF93DF931F92CDB791
:10178000DEB76983DC01ED91FC910280F381E02DED
:1017900041E050E0BE016F5F7F4F09950F90DF91F0
:1017A000CF91089583E08093E9008091F20088232F
:1017B00019F08AE38093E8000895FC0184859585FB
:1017C00097FD0BC09FB7F89482E08093E900809169
:1017D000F2009FBF90E0019608959FB7F89482E0D1
:1017E0008093E9008091F2009FBF90E0089590E01F
:1017F000FC013197EF30F105B0F5EA5AFF4F0C9438
:101800002C27809180008F7703C0809180008F7D8E
:1018100080938000089580918000877FF9CF84B500
:101820008F7702C084B58F7D84BD0895809190002C
:101830008F7707C0809190008F7D03C080919000CA
:10184000877F8093900008958091C0008F7703C0B8
:101850008091C0008F7D8093C00008958091C20068
:10186000877F8093C200089508952E98269A2D9818
:10187000259A2A98229A2998219A80EA80938000B2
:1018800081E18093810080E991E0909387008093CB
:101890008600109289001092880010928B0010929E
:1018A0008A0008954FB141708CB186FB882780F97A
:1018B0008427209171025091700260916B027091A7
:1018C0006C02982F9227292F30E0942F9527291BFF
:1018D0003109260F371F30936C0220936B02209141
:1018E000700290917102821729F0491719F091E066
:1018F00090936F02809370024093710208950E944A
:10190000FC1C90E008950F931F93CF93DF931F92D9
:10191000CDB7DEB78C01FC018485958597FF0EC09D
:10192000CE0101960E94D21C019719F4298130E062
:1019300002C02FEF3FEFF80135872487F801848537
:1019400095850F90DF91CF911F910F910895CF93BF
:10195000DF931F92CDB7DEB7FC018485958597FD97
:1019600005C02FEF3FEF358724870BC0CE010196CE
:101970000E94D21C019719F4898190E002C08FEF78
:101980009FEF0F90DF91CF910895CF93DF93282F92
:1019900030E0F901EE5CFE4F8491F901ED5EFE4FFF
:1019A000D491F901EC50FF4FC491CC2391F08111F7
:1019B0000E94F70BEC2FF0E0EE0FFF1FEA51FF4FF4
:1019C000A591B491EC91ED2381E090E021F480E0C9
:1019D00002C080E090E0DF91CF9108951F93CF93F4
:1019E000DF93282F30E0F901EE5CFE4F8491F9017E
:1019F000ED5EFE4FD491F901EC50FF4FC491CC2322
:101A0000C9F0162F81110E94F70BEC2FF0E0EE0FBA
:101A1000FF1FE852FF4FA591B4918FB7F8941111B1
:101A200005C09C91ED2FE095E92302C0EC91ED2BD0
:101A3000EC938FBFDF91CF911F910895CF93DF93E8
:101A400090E0FC01ED5EFE4F2491FC01EC50FF4F55
:101A50008491882361F190E0880F991FFC01E6537F
:101A6000FF4FC591D491FC01E852FF4FA591B4916D
:101A7000611109C09FB7F8948881209582238883DB
:101A8000EC912E230BC0623061F49FB7F89438813B
:101A9000822F809583238883EC912E2B2C939FBFDC
:101AA00006C08FB7F894E8812E2B28838FBFDF9173
:101AB000CF910895CF93DF93EC01888581110FC0FA
:101AC00081E088878A85882311F062E001C060E0A8
:101AD00089850E941E0D8FE090E00197F1F78985BE
:101AE0000E94C50C2B8530E041E08217930709F472
:101AF00040E0842FDF91CF9108958230910538F036
:101B0000880F991F880F991F05970197F1F708957E
:101B10003FB7F89480917B0290917C02A0917D0266
:101B2000B0917E0226B5A89B05C02F3F19F0019603
:101B3000A11DB11D3FBFBA2FA92F982F8827820F53
:101B4000911DA11DB11DBC01CD0142E0660F771FA3
:101B5000881F991F4A95D1F708958F929F92AF924F
:101B6000BF92CF92DF92EF92FF926B017C010E94B5
:101B7000880D4B015C01C114D104E104F104F1F0C2
:101B80000E94880DDC01CB0188199909AA09BB09BB
:101B9000883E9340A105B10570F321E0C21AD10837
:101BA000E108F10888EE880E83E0981EA11CB11CA4
:101BB000C114D104E104F10419F7DDCFFF90EF90D7
:101BC000DF90CF90BF90AF909F908F9008958F92AD
:101BD0009F92AF92BF92CF92DF92EF92FF920F93BC
:101BE0001F93CF93DF935C016B017A0180912301F6
:101BF000882309F45BC08091D604882309F456C079
:101C00008091800280FF05C08091E0008260809317
:101C1000E000E70110E00AEF83E0882E9AE3992EB6
:101C20002097D9F10E94FC1C81110AC0015009F4CF
:101C30003DC061E070E080E090E00E94AD0DF0CF2B
:101C4000282F30E0C217D3070CF48C2F4FB7F8942D
:101C50008092E9009091E80095FF1DC0282F30E0A8
:101C6000C21BD30BF601982F915020F081918093E5
:101C7000F100FACFC20ED31E112319F09092E800A2
:101C800009C08091E80085FD06C09092E80011E04F
:101C9000209709F010E04FBFC3CF1111C3CF5D985B
:101CA00084E68093D0041E141F0444F081E090E089
:101CB000F5019383828380E090E001C0C701DF914A
:101CC000CF911F910F91FF90EF90DF90CF90BF9039
:101CD000AF909F908F9008957F928F929F92AF9236
:101CE000BF92CF92DF92EF92FF920F931F93CF9309
:101CF000DF93FC0122853385232B09F479C07B0116
:101D0000EC01D12C8C85D816F0F40D2D10E08E85C9
:101D10009F85F801EE0FFF1FEE0DFF1D918380835D
:101D2000EA85FB85E00FF11F61E080810E94EE0CE7
:101D30008A859B85FC01E00FF11F61E080810E9494
:101D40001E0DD394DFCF83E290E00197F1F710E00E
:101D50008C851817A8F4C12ED12CEA85FB85EC0DD3
:101D6000FD1D60E080810E941E0D8A859B85FC011F
:101D7000EC0DFD1D60E080810E94EE0C1F5FE8CF3E
:101D80000E94880D4B015C010E94880DAB01BC01D3
:101D9000481959096A097B098E859F85A0E0B0E042
:101DA000481759076A077B0718F50E94880D6B01D1
:101DB000C818D908712C8C85781630F7072D10E0DB
:101DC000EA85FB85E00FF11F80810E94C50C892BFD
:101DD00051F4000F111FF701E00FF11F8081918175
:101DE000C816D90610F07394E6CFD182C082FBCF1B
:101DF000DF91CF911F910F91FF90EF90DF90CF90E7
:101E0000BF90AF909F908F907F9008952FB7F894D8
:101E100060917702709178028091790290917A02B4
:101E20002FBF08951F920F920FB60F9211242F9378
:101E30003F938F939F93AF93BF938091770290913D
:101E40007802A0917902B0917A023091760223E073
:101E5000230F2D3720F40196A11DB11D05C026E8E2
:101E6000230F0296A11DB11D209376028093770265
:101E700090937802A0937902B0937A0280917B02CA
:101E800090917C02A0917D02B0917E020196A11DED
:101E9000B11D80937B0290937C02A0937D02B0934E
:101EA0007E02BF91AF919F918F913F912F910F90A3
:101EB0000FBE0F901F9018951F920F920FB60F92A2
:101EC00011242F933F934F935F936F937F938F933F
:101ED0009F93AF93BF93EF93FF93E0911201F09123
:101EE00013010995FF91EF91BF91AF919F918F9150
:101EF0007F916F915F914F913F912F910F900FBE06
:101F00000F901F9018951F920F920FB60F921124E9
:101F10002F933F934F935F936F937F938F939F93F1
:101F2000AF93BF93EF93FF93E0911001F0911101F4
:101F30000995FF91EF91BF91AF919F918F917F9103
:101F40006F915F914F913F912F910F900FBE0F9026
:101F50001F9018951F920F920FB60F9211242F9376
:101F60003F934F935F936F937F938F939F93AF9321
:101F7000BF93EF93FF93E0910E01F0910F0109954C
:101F8000FF91EF91BF91AF919F918F917F916F9151
:101F90005F914F913F912F910F900FBE0F901F9027
:101FA00018951F920F920FB60F9211242F933F9303
:101FB0004F935F936F937F938F939F93AF93BF9351
:101FC000EF93FF93E0910C01F0910D010995FF91C2
:101FD000EF91BF91AF919F918F917F916F915F91A1
:101FE0004F913F912F910F900FBE0F901F9018951A
:101FF0001F920F920FB60F9211242F933F934F937E
:102000005F936F937F938F939F93AF93BF93EF9360
:10201000FF93E0910A01F0910B010995FF91EF9177
:10202000BF91AF919F918F917F916F915F914F91F0
:102030003F912F910F900FBE0F901F901895CF9248
:10204000DF92EF92FF920F931F93CF93DF93FC01E8
:102050002081DB018D919C91308552814381A52F98
:10206000B42FA30FB11DA30FB11D4D915C9111971A
:10207000BC01641B750BAB01052E000C660B770BC6
:10208000C184D284E384F4844C0D5D1D6E1D7F1DDC
:1020900041875287638774878D939C938085A6813F
:1020A000B781A80FB11D8C9181110BC02150808583
:1020B000A681B781A80FB11D8C91821708F452C078
:1020C00046C010E09FEF980FF2800381A0856481E5
:1020D0007581492F50E0EB01C40FD51F3881CF2DFA
:1020E000B02FD02FCA0FD11DCA0FD11DAF2DA30FF6
:1020F000B11DA30FB11D0990D881C02D0D90BC91C9
:10210000A02DCA17DB075CF5DB01A80FB11D3C93BE
:10211000A481B581A40FB51F8C91A681B781A80FAA
:10212000B11D8C918F5F8C93808564817581DB01FB
:10213000A40FB51F8C938085A681B781A80FB11D10
:102140008C9181508C9311E0892F9111BBCF8085A8
:102150008F5F8087908189134BC0108649C0111111
:10216000F6CFA4CF90E030E08217930784F7F28097
:102170000381A08564817581AC014F5F5F4FEB01E6
:10218000C40FD51F1881CF2DB02FD02FCA0FD11D4E
:10219000CA0FD11DAF2DA10FB11DA10FB11D099007
:1021A000D881C02D0D90BC91A02DAC17BD077CF639
:1021B000DB01A80FB91F1C93A481B581A40FB51F23
:1021C0008C91A681B781A80FB11D8C9181508C9301
:1021D0008085A481B581A40FB51F8C938085A681CD
:1021E000B781A80FB11D8C918F5F8C93CA01BCCFB2
:1021F0008181A481B581A80FB11D8C912281938129
:10220000E22FF92FE80FF11DE80FF11D8081918178
:10221000DF91CF911F910F91FF90EF90DF90CF90C2
:102220000895CF92DF92EF92FF920F931F93CF9377
:10223000DF93EC018B017A01633071053CF0862F4E
:102240006F3F710521F01CF08FEF01C083E08883A0
:102250006801D594C794C98262E070E0C8010E9409
:102260001C289B838A8361E070E0C8010E941C28BF
:102270009D838C8361E070E0C8010E941C289F83CD
:102280008E83C8860E9DC0010F9D900D1E9D900DE2
:102290001124092E000CAA0BBB0B89879A87AB87E8
:1022A000BC8720E088812817B0F4822F90E0EC8171
:1022B000FD81E80FF91F2083EE81FF81E80FF91FF0
:1022C0002083880F991FEA81FB81E80FF91FF182B3
:1022D000E0822F5FE7CFDF91CF911F910F91FF90A9
:1022E000EF90DF90CF9008950F931F93CF93DF93DC
:1022F0008C01EB0180917502811105C081E0809312
:1023000075020E94350C17FF05C011950195110942
:1023100081E001C080E0013991E0190714F000E983
:1023200011E010938B0000938A00882311F02A9A01
:1023300001C02A98229A80917502811105C081E01E
:10234000809375020E94350CD7FF05C0D195C195C9
:10235000D10981E001C080E0C13991E0D90714F0D2
:10236000C0E9D1E0D0938900C0938800882311F0A0
:10237000299A01C02998219ADF91CF911F910F913D
:10238000089546983E9AE0E9F0E082E0808310925A
:102390009100109271001082109299001092980092
:1023A000109297001092960010929500109294004F
:1023B00086988E980895FC01109271009B01461733
:1023C000570708F49A0146983E9890E89093900039
:1023D00010929100909392003E9AEF2B11F08E9AFA
:1023E00001C08E98869A5093970040939600415072
:1023F0005109509395004093940030939900209395
:10240000980082E88093900089E18093910008957C
:1024100024982C9A6A98729A6E98769A8098889ADC
:1024200081E08093680090E190936B008BBB82E524
:102430009CE09093130180931201EAE6F0E0808122
:102440008F7C80618083EE9A8CB182FB882780F933
:102450008093740293B12091740294FB882780F9D1
:1024600082278093730210926E0210926D02109276
:1024700072028FB18170809371029CB120917102C0
:1024800096FB882780F982278093700210926C0255
:1024900010926B0210926F0208951F920F920FB666
:1024A0000F9211242F933F934F935F936F937F93DA
:1024B0008F939F938CB190E095958795959587958F
:1024C000482F417023B130E054E0359527955A9557
:1024D000E1F7822793278170209174025091730253
:1024E00060916D0270916E02982F9227292F30E033
:1024F000942F9527291B3109260F371F30936E0221
:1025000020936D022091730290917402821729F03A
:10251000491719F091E090937202809373024093EF
:1025200074029F918F917F916F915F914F913F9135
:102530002F910F900FBE0F901F9018951F93CF9360
:10254000DF930E94E902C0E0D0E01AE090ED980F1E
:102550009A30B8F41C9F90011D9F300D1124E901A1
:10256000C80FD11D87FDDA95E0978091690290919F
:102570006A02019690936A02809369020E94E902BE
:10258000E5CFCE01DF91CF911F9108950E942F2AB0
:102590004091C4042091C2043091C30490E0941788
:1025A00049F02D5F3F4FF90133975081581721F0C3
:1025B0009F5FF5CF8FEF0895892F08952091140321
:1025C0009091CF04213208F04AC08091F10281112C
:1025D000FCCF32E03093F10231E03093F0023FEF74
:1025E0003093EF021092EE022093ED02A4EFB2E0DE
:1025F0004DEC52E0FA013E2F341B321718F43D9196
:102600003193F9CF1092CC022091CC02990F922BEA
:102610009093CC029091CB02913061F41092CB0256
:102620009091CC029093BB009091BC0093FDF8CFA9
:1026300095EC01C095EE9093BC009091F102923020
:10264000E1F39091EF029F3F79F08091EF028032A9
:1026500041F08091EF02803331F084E005C081E0E9
:1026600003C082E001C083E01092F30210921403D1
:102670001092F202089591E09093F2028093CF04B9
:102680001092F3021092140308959091F1029111A7
:10269000FCCF613208F060E291E09093F1029093F8
:1026A000F0022FEF2093EF021092EE02260F2093FC
:1026B000ED029093CC029091CC02880F892B8093ED
:1026C000CC028091CB02813061F41092CB028091D8
:1026D000CC028093BB008091BC0083FDF8CF85ECD9
:1026E00001C085EE8093BC008091F1028130E1F35E
:1026F0008091EE02861710F46091EE02ADECB2E02C
:102700002BEA32E0F9018E2F821B861718F48D9187
:102710008193F9CF1092AA026093A902862F08959F
:10272000CF93C82F0E943B136FE082E094E00E9499
:10273000B6020E94DE1281110FC061E08C2F0E9450
:1027400045139091A9028091AA02981729F082E07E
:1027500094E0CF910C946A028FEF9FEFCF91089590
:10276000BF92CF92DF92EF92FF920F931F93CF937E
:10277000DF93809172040E943B1368EA82E094E048
:102780000E94B6020E94DE1266E0809172040E94EE
:1027900045130E94060F7B018091A90290E02091D1
:1027A000AA02821B91090697ACF480917304909160
:1027B0007404892B89F30E94060F6E197F0980919A
:1027C0007304909174048617970730F781E0809323
:1027D000750433C082E094E00E946A02C82E82E051
:1027E00094E00E946A02B82E82E094E00E946A029D
:1027F000E82E82E094E00E946A02D82E82E094E003
:102800000E946A02F82E82E094E00E946A021B2D68
:1028100000E00C2910936A0400936904DD2D20E088
:10282000C22FCE29D0936C04C0936B04982F8827B5
:102830008F2990936E0480936D04DF91CF911F9147
:102840000F91FF90EF90DF90CF90BF9008950F937E
:102850001F93CF93DF93082F162FC9E6D4E0898505
:102860000E943B13602F82E094E00E94B602612F29
:1028700082E094E00E94B6020E94DE128E83DF9115
:10288000CF911F910F910895CF93DF93BC0182EBFD
:1028900093E00E94811AEC016DE072E082EB93E01C
:1028A0000E94811A8C0F9D1FDF91CF9108958BE6B6
:1028B0000E9490138F3F2FEF920781F48AE60E94C7
:1028C00090138F3F2FEF920761F489E60E949013D7
:1028D000833D910541F521E030E02DC021E030E05D
:1028E00002C020E030E0873D9105D1F081E090E02A
:1028F00090937104809370040197029738F421300B
:10290000310511F08AE608C08BE606C0213031059A
:1029100011F088E601C089E68093720481E0089591
:1029200082E090E0E5CF88E60E949013833D910518
:1029300029F420E030E080E090E0DACF80E00895F4
:10294000EF92FF920F931F93CF93DF9380919204A6
:102950000E943B1380918F0490919004039731F46F
:102960006091970470919804606804C06091950428
:102970007091960482E094E00E94B6020E94DE12FA
:1029800080938E0466E0809192040E9445130E9419
:10299000060FEB018091A90290E02091AA02821B10
:1029A00091090697ACF48091A1049091A204892B1F
:1029B00089F30E94060F6C1B7D0B8091A1049091FE
:1029C000A2048617970730F781E08093A30474C0B0
:1029D00080918F04909190040397F9F482E094E041
:1029E0000E946A02182F82E094E00E946A02E82E98
:1029F00082E094E00E946A02D82F82E094E00E9474
:102A00006A02F82E82E094E00E946A02C82F82E0F7
:102A100094E00E946A02082F39C082E094E00E948C
:102A20006A02E82E82E094E00E946A02182F8091E8
:102A30008F0490919004892BA9F482E094E00E9485
:102A40006A02F82E82E094E00E946A02D82F82E0A7
:102A500094E00E946A02082F82E094E00E946A02D9
:102A6000C82F14C082E094E00E946A02082F82E01E
:102A700094E00E946A02C82F82E094E00E946A02F9
:102A8000F82E82E094E00E946A02D82F212F30E0D5
:102A90003E2930937D0420937C042D2F30E03F2984
:102AA00030937F0420937E042C2F30E0C901902BBB
:102AB0009093810480938004DF91CF911F910F91B7
:102AC000FF90EF900895BF92CF92DF92EF92FF9226
:102AD0000F931F93CF93DF93809191040E943B1338
:102AE00068EA82E094E00E94B6020E94DE128093BF
:102AF0008E0466E0809191040E9445130E94060FA7
:102B00007B018091A90290E02091AA02821B910989
:102B10000697ACF48091A1049091A204892B89F3CB
:102B20000E94060F6E197F098091A1049091A20462
:102B30008617970730F781E08093A30433C082E0C3
:102B400094E00E946A02C82E82E094E00E946A0229
:102B5000B82E82E094E00E946A02E82E82E094E0BF
:102B60000E946A02D82E82E094E00E946A02F82E47
:102B700082E094E00E946A021B2D00E00C29109371
:102B8000770400937604DD2D20E0C22FCE29D09368
:102B90007904C0937804982F88278F2990937B0419
:102BA00080937A04DF91CF911F910F91FF90EF9066
:102BB000DF90CF90BF9008950F931F93CF93DF9333
:102BC000082F162FC6E7D4E08C8D0E943B13602F90
:102BD00082E094E00E94B602612F82E094E00E94BD
:102BE000B6020E94DE12888FDF91CF911F910F9164
:102BF00008950F931F93CF93DF93082F162FC6E7E7
:102C0000D4E08B8D0E943B13602F82E094E00E9401
:102C1000B602612F82E094E00E94B6020E94DE12AA
:102C2000888FDF91CF911F910F91089520918F048C
:102C3000309190042330310511F0803210F40C945F
:102C4000DC150C94F9151F93CF93DF931F92CDB72A
:102C5000DEB7182F69830E943B13698182E094E0FC
:102C60000E94B6020E94DE12811112C061E0812F23
:102C70000E9445139091A9028091AA02981741F0F1
:102C800082E094E00F90DF91CF911F910C946A0243
:102C90008FEF9FEF0F90DF91CF911F91089540919B
:102CA000D3045091D4042091D1043091D20442171E
:102CB0005307B4F49091E8009570E1F39091E80027
:102CC00092FD19C08093F1008091D3049091D404B7
:102CD00001968F739927892B19F48EEF8093E80062
:102CE0008091D3049091D40401969093D40480935E
:102CF000D30481E0089580E00895DF92EF92FF927F
:102D00000F931F93CF93DF93D82E8A017B01E40E9C
:102D1000F51EEB01CE15DF0571F0D7FE03C0FE01F5
:102D2000849101C088810E944F1621968111F2CFB3
:102D30008FEF9FEF01C0C801DF91CF911F910F91DD
:102D4000FF90EF90DF900895615030F02091F100F6
:102D5000FC0120830196F8CF289884E68093D5045F
:102D60000895CF92DF92EF92FF920F931F93CF932C
:102D7000DF936C017A018B01C0E0D0E0CE15DF0556
:102D800089F0D8016D918D01D601ED91FC910190F2
:102D9000F081E02DC6010995892B11F47E0102C056
:102DA0002196ECCFC701DF91CF911F910F91FF903A
:102DB000EF90DF90CF900895FC01538D448D252F27
:102DC00030E0842F90E0821B930B541710F0CF96C5
:102DD000089501970895FC01918D828D981761F0F7
:102DE000828DDF01A80FB11D5D968C91928D9F5F42
:102DF0009F73928F90E008958FEF9FEF0895FC01ED
:102E0000918D828D981731F0828DE80FF11D858D9F
:102E100090E008958FEF9FEF0895FC01918D228D32
:102E2000892F90E0805C9F4F821B91098F739927B7
:102E3000089585E193E00E940D1721E0892B09F4A4
:102E400020E0822F0895FC01848DDF01A80FB11DC1
:102E5000A35ABF4F2C91848D90E001968F739927D0
:102E6000848FA689B7892C93A089B1898C918064BD
:102E70008C93938D848D981306C00288F389E02D7E
:102E800080818F7D80830895EF92FF920F931F932F
:102E9000CF93DF93EC0181E0888F9B8D8C8D98130D
:102EA00005C0E889F989808185FD24C0F62E0B8D47
:102EB00010E00F5F1F4F0F731127E02E8C8DE8126B
:102EC0000CC00FB607FCFACFE889F989808185FF2D
:102ED000F5CFCE010E942317F1CF8B8DFE01E80FB5
:102EE000F11DE35AFF4FF0820B8FEA89FB89808145
:102EF000806207C0EE89FF896083E889F989808153
:102F00008064808381E090E0DF91CF911F910F91E9
:102F1000FF90EF900895CF93DF93EC01888D882385
:102F2000C9F0EA89FB89808185FD05C0A889B98936
:102F30008C9186FD0FC00FB607FCF5CF808185FF11
:102F4000F2CFA889B9898C9185FFEDCFCE010E947F
:102F50002317E7CFDF91CF9108950F931F93CF935E
:102F6000DF931F92CDB7DEB782E0898342E450E061
:102F700061E571E080E80E947D160E940D1DDC0174
:102F800012960D911C9113970115110569F0D80146
:102F9000ED91FC910280F381E02DBE016F5F7F4FC8
:102FA000C801099597FF07C089810F90DF91CF91E4
:102FB0001F910F910895F80100851185E5CF1F92AB
:102FC0000F920FB60F9211248F939F938091E1007F
:102FD0009091E100937F9093E10083FF0FC01092E6
:102FE000E90091E09093EB001092EC0092E3909353
:102FF000ED001092D60498E09093F00082FF20C07C
:1030000093E09093E9009091F200992319F09AE3EC
:103010009093E8009091D004992339F09091D004D6
:1030200091509093D004992389F19091D5049923DC
:1030300039F09091D50491509093D504992341F1A2
:1030400084FF10C08091E2008E7E81608093E20058
:103050008091E1008F7E8093E100809180028E7EDE
:10306000806111C080FF16C08091E2008E7E806179
:103070008093E2008091E1008E7E8093E100809158
:1030800080028E7E81608093800204C05D9ACDCFE5
:10309000289AD6CF9F918F910F900FBE0F901F90BF
:1030A00018951F920F920FB60F921124CF92DF92B4
:1030B000EF92FF920F931F932F933F934F935F9342
:1030C0006F937F938F939F93AF93BF93EF93FF93F0
:1030D000CF93DF93CDB7DEB76C97DEBFCDBF109235
:1030E000E9008091E80083FFEDC168E0CE014596DC
:1030F0000E94A41682EF8093E8008D8987FF05C0A7
:103100009091E80090FFFCCF03C09EEF9093E80001
:10311000982F907609F0C6C09E892F89188D91113D
:103120000CC0803829F4809181028093F10002C0A4
:103130001092F1001092F10048C1422F50E0512B43
:10314000913051F4811141C14130510509F03DC127
:10315000809181028D7F0BC0933061F4811135C164
:103160004130510509F031C1809181028260809324
:1031700081022BC1953041F48091E80080FFFCCFA3
:1031800020682093E30021C1963009F05FC0EB8CEA
:10319000FC8C1092E9001092D4041092D3041230E7
:1031A00091F51092D2041092D1040E94AD1799E0CB
:1031B000BE016F5F7F4FDB01E92F1D92EA95E9F7B2
:1031C00099831A8391E09E8390EA98879AEF998772
:1031D0002091D3043091D404275F3F4F3C832B834D
:1031E0008D831092E9001092D4041092D304F092CF
:1031F000D204E092D10449E050E080E00E947D16C4
:103200000E94AD17E2C0F092D204E092D1040E9475
:103210000D1DDC011296ED90FC901397E114F10462
:1032200009F4C0C0D701ED91FC910480F581E02D37
:10323000BE016B5E7F4FC7010995009719F00CF036
:10324000C4C0C7C0F701E084F184E8CF973009F427
:10325000C0C0983021F481E08093F100B6C099306D
:1032600009F0B3C0837009F0B4C0EDEAF1E081E089
:1032700021E036E39081992361F08093E900209367
:10328000EB0091919093EC003093ED008F5F8730CD
:1032900089F78EE78093EA001092EA008F89809385
:1032A000D60493C08B8D9C8D1092E9001092D404AB
:1032B0001092D3049093D2048093D104898D81110C
:1032C00056C08E899D89913A59F4813209F081C0A6
:1032D00047E050E06CE171E080E00E947D1675C02F
:1032E000913209F076C0833289F4888D90E0982F6E
:1032F00088272F89822BA0E0B0E08093180190935B
:103300001901A0931A01B0931B015FC0803269F4C8
:103310008091E80082FFFCCF67E08CE191E00E94A1
:10332000A4168BEF8093E80006C0823209F04DC0EE
:103330008F898093230180917F02882319F0EEEF1B
:10334000FAE002C0E0E0F8E080911C0190911D01DC
:10335000A0911E01B0911F01803B9440A105B105D1
:1033600009F07BC08091230180FF93C076C00E944A
:103370000D1DDC0112960D911C911397011511057D
:1033800041F1D801ED91FC910190F081E02DBE0159
:103390006B5E7F4FC8010995811117C0F801008548
:1033A0001185ECCF113009F44EC0133091F48F89A0
:1033B000882309F445C0823081F440E860E185EB60
:1033C00091E00E94BC24882321F08EEF8093E800D6
:1033D00079C081E28093EB0075C0813029F440E828
:1033E0006BE089EA91E0EDCF833099F70E940D1DE3
:1033F000DC011296ED90FC9013978E010F5F1F4F2A
:103400006801E114F10479F0D701ED91FC91068097
:10341000F781E02DB801C7010995080F111DF701CB
:10342000E084F184EECFD8011C92F60101900020D7
:10343000E9F73197BF016C197D0940E0C601C1CFA2
:1034400063E971E002C067E971E06115710509F295
:10345000FB01449150E080E840CF0FB6F894A89566
:1034600080916000886180936000109260000FBEC0
:10347000A895EE3F2AE0F20739F08091FE0A90917C
:10348000FF0A91838083A1CF1092FF0A1092FE0A57
:103490009CCFEE3F8AE0F80731F0808191819093D4
:1034A000FF0A8093FE0A87E797E7918380839BE07A
:1034B00088E10FB6F894A895809360000FBE9093B2
:1034C000600083CF6C960FB6F894DEBF0FBECDBF01
:1034D000DF91CF91FF91EF91BF91AF919F918F912C
:1034E0007F916F915F914F913F912F911F910F911C
:1034F000FF90EF90DF90CF900F900FBE0F901F9036
:1035000018956115710579F0FB0101900020E9F72C
:103510003197AF01461B570BDC01ED91FC91028006
:10352000F381E02D099480E090E008951F920F92BE
:103530000FB60F9211242F933F934F935F936F9386
:103540007F938F939F93AF93BF93EF93FF9385E107
:1035500093E00E942317FF91EF91BF91AF919F914C
:103560008F917F916F915F914F913F912F910F902C
:103570000FBE0F901F9018951F920F920FB60F92CB
:1035800011242F938F939F93EF93FF93E091250343
:10359000F09126038081E0912B03F0912C0382FDB2
:1035A00012C0908180912E038F5F8F7320912F0323
:1035B000821751F0E0912E03F0E0EB5EFC4F958F07
:1035C00080932E0301C08081FF91EF919F918F9195
:1035D0002F910F900FBE0F901F9018958091BD04F2
:1035E0008F3F61F061E00E941E0D60E08091BD049C
:1035F0000E94EE0C8BE193E00197F1F708956FE0E4
:1036000070E08DE10E9423168934910561F06FE02E
:1036100070E08EE10E9423168934910509F0A2C062
:1036200020E030E002C021E030E083E090E09093C1
:10363000900480938F048230910539F589E180935D
:1036400091048EE18093920483E090E0909396043D
:103650008093950484E090E090939804809397047D
:1036600087E090E090939A048093990488E090E03A
:1036700090939C0480939B0485E090E090939E043B
:1036800080939D0486E090E030C08330910599F1ED
:10369000019709F45FC02130310509F461C088E168
:1036A000809391048EE18093920483E090E0909364
:1036B00096048093950484E090E09093980480931E
:1036C000970485E090E090939A048093990486E0B3
:1036D00090E090939C0480939B0487E090E090930B
:1036E0009E0480939D0488E090E09093A0048093D2
:1036F0009F0481E008952130310511F08EE101C071
:103700008DE1809392048093910488E090E09093FF
:1037100098048093970489E090E0909396048093B6
:1037200095048AE090E090939C0480939B048BE046
:1037300090E090939A04809399048CE090E09093A9
:10374000A00480939F048DE090E090939E0480936A
:103750009D04CFCF2130310509F470CF88E16FCFC0
:1037600089E19ECF60E270E089E10E942316019614
:1037700061F06FE070E08EE10E94231621E030E0FE
:10378000CC97D9F080E090E052CF60E270E088E121
:103790000E942316019679F06FE070E08EE10E949E
:1037A000231631E020E0CC9709F030E0832F922FF0
:1037B00020E030E03CCF80E0089582E090E037CF19
:1037C000FF920F931F93CF93DF93CDB7DEB7A097F0
:1037D0000FB6F894DEBF0FBECDBF8C01F62E8FEF73
:1037E000860F823088F48091BD048F3F79F061E0CC
:1037F0000E941E0D61E08091BD040E94EE0C8BE1E1
:1038000093E00197F1F702C00E94EE1AE091B00434
:10381000F091B1040190F081E02DB80180EB94E0CB
:1038200009950E94EE1A62E0F61231C0E091B004F0
:10383000F091B1040190F081E02DBE016F5F7F4FE8
:1038400080EB94E0099540E08091BC044817F8F4BF
:10385000242F30E0220F331FF801E20FF31FA1E005
:10386000B0E0AC0FBD1FA20FB31F8091BE049091BA
:10387000BF042D913C91BC01621B730B9B018081A5
:103880009181280F391F318320834F5FDDCFA096B0
:103890000FB6F894DEBF0FBECDBFDF91CF911F9161
:1038A0000F91FF9008958F929F92AF92BF92CF9207
:1038B000DF92EF92FF920F931F93CF93DF93CDB7D9
:1038C000DEB7A1970FB6F894DEBF0FBECDBF6C0177
:1038D000990FEE08FF08F7FE33C0E0911503F09151
:1038E00016030190F081E02D6DE285E193E00995EA
:1038F0008C0122273327A9012C193D094E095F09A4
:1039000019A2CE0181967C019AE0892E912CA12CDE
:10391000B12CCA01B901A50194010E940F26605D76
:10392000F70162937F01211531054105510589F7A2
:10393000BF0185E193E00E94811A800F911F1FC093
:10394000A701960119A28E010F5D1F4F8AE0C82EB4
:10395000D12CE12CF12CCA01B901A70196010E94DA
:103960000F26605DF80162938F0121153105410535
:10397000510589F7BF0185E193E00E94811AA19664
:103980000FB6F894DEBF0FBECDBFDF91CF911F9170
:103990000F91FF90EF90DF90CF90BF90AF909F90EE
:1039A0008F900895FC018091D604811103C08FEFA0
:1039B0009FEF08959FB7F89482E08093E9002091EB
:1039C000F20030E01216130614F421E030E0211565
:1039D000310559F0289884E68093D5048091F10050
:1039E00080838091F200882319F09FBFC901089558
:1039F0008BE68093E800F9CF2FB7F89483E08093AB
:103A0000E9009091E800892F807295FF04C09091A1
:103A1000F20080E4891B2FBF08958091DB0481119F
:103A20000DC082E08093D70484E08093D804109284
:103A3000DA041092D90481E08093DB0487ED94E0EE
:103A4000089584EA91E09093B1048093B00480914A
:103A5000BA049091BB04009711F00E94CD28809188
:103A6000B4049091B504009711F00E94CD28809184
:103A7000B8049091B904009711F00E94CD2880916C
:103A8000B2049091B304009711F00E94CD28809168
:103A9000B6049091B704009711F00C94CD280895C6
:103AA000CF93DF93CDB7DEB7CB56D1090FB6F894DD
:103AB000DEBF0FBECDBF789484B5826084BD84B56F
:103AC000816084BD85B5826085BD85B5816085BD19
:103AD00080916E00816080936E00109281008091D1
:103AE0008100826080938100809181008160809359
:103AF000810080918000816080938000809191009E
:103B00008260809391008091910081608093910008
:103B1000809190008160809390008091C1008460CA
:103B20008093C1008091C10082608093C100809128
:103B3000C10081608093C1008091C3008160809347
:103B4000C3008091C00082608093C0008091C20059
:103B500081608093C20080917A00846080937A00B3
:103B600080917A00826080937A0080917A008160EF
:103B700080937A0080917A00806880937A00109216
:103B8000D60410928102109280028091D700816049
:103B90008093D70080EA8093D80089B5806189BD81
:103BA00089B5826089BD09B400FEFDCF61E070E097
:103BB00080E090E00E94AD0D8091D8008F7C806104
:103BC0008093D8008091E000807F8093E000809116
:103BD000E1008E7E8093E1008DE08093E200559AB3
:103BE000209AEEEFFFE7859194918B3F9C4D19F45D
:103BF00081E080937F02E0912503F091260382E02B
:103C00008083E0912103F09122031082E09123034D
:103C1000F09124038FEC808310922D03E09129030F
:103C2000F0912A0386E08083E0912703F091280336
:103C3000808180618083E0912703F0912803808157
:103C400088608083E0912703F09128038081806859
:103C50008083E0912703F091280380818F7D80830A
:103C60008AE090E0A0E0B0E08093190390931A03FB
:103C7000A0931B03B0931C0385E193E00E940D17F2
:103C8000892B21F083EB91E00E94441485E193E0BD
:103C90000E940D171816190624F485E193E00E947E
:103CA000EB161092AA021092A9021092F30210923F
:103CB00014031092F10281E08093F0021092CB0283
:103CC00061E082E00E94EE0C61E083E00E94EE0C75
:103CD0008091B9008E7F8093B9008091B9008D7F6B
:103CE0008093B90088E48093B80085E48093BC0099
:103CF00064EF71E080E090E00E94AD0D8BE0809376
:103D0000C50469E070E08091C2049091C3040E94F0
:103D10006529FC01009769F09093C3048093C20465
:103D200083E08093C40484E1808386E1838384E01C
:103D3000868381E00E94CC0882E1898385E18A83C1
:103D40008CE08B831092B3041092B2041092B504ED
:103D50001092B4041092B7041092B6041092B904F1
:103D60001092B8041092C1041092C00483E08093B2
:103D7000BC048091BA049091BB04892B11F080E0BF
:103D80000BC083E090E00E9438289093BB0480939E
:103D9000BA04892BA1F719C09091BC04891790F43B
:103DA000282F30E0E091BA04F091BB04E20FF31F3A
:103DB000A1E0B0E0AC0FBD1FA20FB31F9C91908398
:103DC0008F5FEACF8BE08093BD0480ED97E0909306
:103DD000BF048093BE0431EEA2963FAFA297412C60
:103DE000512C3201812C912C5401C12CD12C760103
:103DF000A2964FADA2974C3328F46CE97FEF88E68A
:103E000090E004C064E670E088E99FEF0E947411BE
:103E100061E082E892E00E94E01B80918202909132
:103E20008302C80ED91EE11CF11C8091840290917E
:103E30008502880E991EA11CB11C8091860290916A
:103E40008702480E591E611C711C8091B404909128
:103E5000B504892B39F08091B2049091B304892B79
:103E6000D1F41CC00091BC0410E0C801880F991F58
:103E70000E9438289093B5048093B404009709F405
:103E8000C5C0FC0180E090E08017910724F71192F3
:103E900011920196F9CF00E010E01DC00091BC0422
:103EA00010E0C801880F991F0E9438289093B3042E
:103EB0008093B204009709F4A9C02091BE04309108
:103EC000BF04FC0180E090E08017910724F7219364
:103ED00031930196F9CF61E0CE018F5B9F4F0E9435
:103EE000E01B8091BC04A82FB0E0A696BFAFAEAF98
:103EF000A697FE013196A496FFAFEEAFA497E05CC3
:103F0000FF4F9E012F5D3F4F1901AC963FAF2EAF83
:103F1000AC97AE014F5F5F4F60E070E0A6968EAD4C
:103F20009FADA69768177907BCF501151105A1F09B
:103F3000AC96AEADBFADAC972D913C918081918197
:103F40002817390748F0DA012D913C918081918141
:103F50008217930760F010C080819181AC96AEAD5E
:103F6000BFADAC978D939C930115110561F78081CE
:103F70009181DA018D939C936F5F7F4F4E5F5F4F0E
:103F80003296AC962EAD3FADAC972E5F3F4FAC96C0
:103F90003FAF2EAFAC97C2CF0F5F1F4F0A30110556
:103FA00009F099CFA091B204B091B3046091B40428
:103FB0007091B50480E090E02091BC0430E082175D
:103FC000930724F5A496EEADFFADA497219131910E
:103FD000A496FFAFEEAFA497FB0140815181421739
:103FE000530710F431832083F101219131911F0196
:103FF0004D915C9111972417350718F411963C9355
:104000002E93019612966E5F7F4FD6CFA2962FAD5C
:10401000A2972F5FA2962FAFA297293509F0E8CE7D
:1040200060E070E080E090E00E947411C701B6018A
:1040300028E730E040E050E00E940F2630938302F2
:1040400020938202C501B40128E730E040E050E04F
:104050000E940F263093850220938402C301B2018F
:1040600028E730E040E050E00E940F2630938702BE
:104070002093860280E00E94CC0881E00E94CC0858
:104080000E9457140E94571481110DC02898209A3D
:1040900083ED91E00E94441468E873E180E090E0D1
:1040A0000E94AD0DF5CF6FEF80E20E94271460E211
:1040B00083E20E94271460E084E20E94271400E05B
:1040C00014E0C12CD12C7601809172040E943B1324
:1040D00067E282E094E00E94B6020E94DE128093C2
:1040E0006F0461E0809172040E94451382E094E0C5
:1040F0000E946A020E94DE120E94B01380916D0439
:1041000090916E04092E000CAA0BBB0BC80ED91E91
:10411000EA1EFB1E01501109B9F6C701B60120E0E5
:1041200034E040E050E00E94A62530938B022093BB
:104130008A020E94880D709389026093880280E051
:104140000E94CC0881E00E94CC080E94FF1A0E94C5
:10415000FF1A81110DC02898209A8FEE91E00E94DD
:10416000441468E873E180E090E00E94AD0DF5CF63
:1041700080918F049091900483309105A9F460E0C0
:1041800081E20E94161667E580E20E94161664E638
:1041900084E20E94161660E285E20E94161660E034
:1041A00086E20E9416161CC0029731F468E083E292
:1041B0000E94F91567E405C060E083E20E94F915EA
:1041C00067E280E20E94F9156CE080E00E94DC1555
:1041D00060E281E00E94DC1560E082E00E94DC1574
:1041E00000E014E060E070E0CB01A7966FAFA79706
:1041F000A8967FAFA897A9968FAFA997AA969FAFC9
:10420000AA970E9463150E94A014C0907604D090D3
:1042100077040D2C000CEE08FF08A7966FADA7974A
:10422000A8967FADA897A9968FADA997AA969FAD9E
:10423000AA976C0D7D1D8E1D9F1D01501109A9F6B9
:1042400020E034E040E050E00E94A6253093A30235
:104250002093A20280E00E94CC085D98559AE091DC
:10426000A404F091A5040190F081E02D84EA94E08B
:1042700009958823A1F36AE070E080E090E00E9455
:10428000AD0DE091A404F091A5040190F081E02D22
:1042900084EA94E00995882311F3E091A404F09155
:1042A000A5040190F081E02D84EA94E00995811144
:1042B000F4CF6AE070E080E090E00E94AD0DE09104
:1042C000A404F091A5040190F081E02D84EA94E02B
:1042D00009958111E2CF0E94060F611571058105D4
:1042E000910511F00E944C2564EF71E080E090E0B0
:1042F0000E94AD0D11E0C12CD12C80E8E82E8FE397
:10430000F82E93E3892E982C93EBA92E9FE3B92ED8
:104310005D9A559A80E00E94CC08289A209A0E94C3
:104320003F070E9434060E946B060E9463150E949C
:10433000A01480917604909177042091A20230918C
:10434000A302821B930B9093A5028093A4020E9468
:10435000E0060E94BF0885E193E00E940D17181641
:10436000190644F485E193E00E94EB169093A802AD
:104370008093A7028091A7029091A80281339105B2
:1043800019F41093A60204C0C09711F41092A6026B
:104390008091A6028823A1F18092140190921501C8
:1043A000A0921601B09217018091A4029091A502EB
:1043B0008D3D9540ECF480919F02863021F48091F0
:1043C000A0028630A9F08091980290919902853FD1
:1043D000914074F480919C0290919D02853F9140A0
:1043E0003CF480919A0290919B02853691052CF0C5
:1043F00060E070E080E090E085C10E94D308E1C1F8
:10440000C0921401D0921501E0921601F0921701AA
:1044100080919F02863009F078C18091A002863099
:1044200009F073C181E090E00E94531C81E00E947A
:10443000CC08109290021092910210929202109267
:10444000930210928C0210928D0210928E021092A2
:104450008F020E946B0680918C0290918D02A09138
:104460008E02B0918F024497A105B1055CF40E94C1
:104470006B060E94E00664E670E08AE190E00E942C
:104480007411E9CF0E946B0680918C0290918D028D
:10449000A0918E02B0918F028D97A105B1059CF479
:1044A0000E946B060E94E00664E670E08AE190E0FC
:1044B0000E94741180919C0290919D0289579109EC
:1044C0008B37914008F70E94E00680919C02909102
:1044D0009D02883791054CF40E94E00664E670E086
:1044E00088E690E00E947411F0CF0E946B068091E4
:1044F0008C0290918D02A0918E02B0918F020B9749
:10450000A105B1051CF10E946B060E94E006809196
:10451000980290919902875991098D35914018F42C
:1045200060E070E00EC080919C0290919D028957DE
:1045300091098B37914018F464E670E002C069E19C
:1045400070E088E690E00E947411D1CF64E670E0DC
:1045500088E690E00E9474110E943F070E94060FB7
:1045600070939702609396028091A102863078F44E
:104570000E943F070E94E0060E94D3080E94BF08E5
:104580008091940290919502893B9B4068F30E9430
:104590003F078091A102863039F40E943F070E94B4
:1045A000E0060E94D308F5CF0E94060F7093970291
:1045B000609396020E94BF088091940290919502A8
:1045C000883B9B4028F40E94E0060E94D308F2CF6B
:1045D0001092900210929102109292021092930205
:1045E00010928C0210928D0210928E0210928F0205
:1045F0000E946B0680918C0290918D02A0918E0298
:10460000B0918F028D3E9F4FAF4FBF4F5CF00E9425
:104610006B060E94E00669E170E088E690E00E9487
:104620007411E8CF0E946B0680918C0290918D02EC
:10463000A0918E02B0918F02843D9F4FAF4FBF4F2C
:104640009CF00E946B060E94E00669E170E088E63B
:1046500090E00E947411809198029091990287597C
:1046600091098D35914000F70E94E00680919802F3
:1046700090919902863991054CF40E94E00664E617
:1046800070E088E690E00E947411F0CF0E946B0603
:1046900080918C0290918D02A0918E02B0918F0238
:1046A000863F9F4FAF4FBF4F2CF50E946B060E9475
:1046B000E00680919C0290919D02895791098B3769
:1046C000914028F464E670E080E090E010C08091B2
:1046D0009802909199028759910964E670E08D35AE
:1046E000914018F488E690E002C08AE190E00E94D0
:1046F0007411CECF80E090E00E94531C64E670E01D
:1047000088E690E00E9474115CC02091980230917C
:104710009902255F314080919A0290919B022B343F
:10472000344048F49C012D523140233F314018F46D
:104730000E94B10946C020919C0230919D02255FE4
:1047400031402B34344030F49C012D523140233F12
:10475000314070F385569109873C910508F04DCEA4
:104760002898209A81E090E00E94531C0E94060F36
:1047700070939702609396028091980290919902AB
:10478000863991052CF080E090E00E94531C19C0FE
:1047900080919C0290919D0288379105A4F70E9418
:1047A000BF080E94E0066CE97FEF88E99FEF0E9456
:1047B00074118091940290919502893B9B40E0F2A4
:1047C000E2CF0E94B20BA4CDE5E1F3E013821282A6
:1047D00088EE93E0A0E0B0E084839583A683B7835E
:1047E00022E631E0318320832DEC30E035872487C9
:1047F0002CEC30E03787268728EC30E0318B208B9B
:1048000029EC30E0338B228B2AEC30E0358B248B83
:104810002EEC30E0378B268B118E128E138E148E79
:10482000E2EBF3E01382128284839583A683B7833D
:1048300024E731E0318320832FEF3FEF3587248752
:10484000E2E0F4E01382128284839583A683B78327
:1048500086E891E091838083E2ECF4E0118210829B
:1048600012828FEF838315821482168285EA91E08B
:104870009287818782E492E09487838784EA91E03B
:1048800090878783E0EBF4E0138212821582148212
:104890001782168211861086138612868AEA91E0A4
:1048A00091838083E4EAF4E01282158210868EE020
:1048B000818781E08287838788E991E09183808383
:1048C00086E0E2E5F1E0A8E8B4E001900D928A9577
:1048D000E1F786E0E8E5F1E0A2E8B4E001900D92AE
:1048E0008A95E1F7E6E7F4E084E090E0928F818F2B
:1048F00014A613A615A6E9E6F4E083E090E09087FD
:10490000878313861286148640E050E063E070E0EF
:104910008CE594E00E94111140E050E063E070E00B
:104920008FE494E00E94111140E050E063E070E0F9
:1049300082E494E00E94111140E050E063E070E0F6
:1049400085E394E00E94111140E050E063E070E0E4
:1049500088E294E00E94111140E050E063E070E0D2
:104960008BE194E00E94111140E050E063E070E0C0
:104970008EE094E00C941111CF92DF92EF92FF92AF
:104980000F931F93CF93DF931F92CDB7DEB7182FEE
:10499000062FE42E862F880F8E5F99830E944F1674
:1049A00083E00E944F16F12EC12E9981D92E8C2DB5
:1049B0008F19801798F4F601E7FE02C0849101C0B8
:1049C00080810E944F16182F80E00E944F1681238D
:1049D000FFEFCF1ADF0A8111EACF01C081E00F900B
:1049E000DF91CF911F910F91FF90EF90DF90CF90CB
:1049F00008958F929F92AF92BF92CF92DF92EF92E3
:104A0000FF92CF93DF93EC01688179818A819B814A
:104A1000611571058105910521F464E279ED8BE55D
:104A200097E02DE133EF41E050E00E94A6254901D7
:104A30005A019B01AC01A7EAB1E40E94C5256B01B4
:104A40007C01ACEEB4EFA50194010E94D325DC01FA
:104A5000CB018C0D9D1DAE1DBF1DB7FF03C001977F
:104A6000A109B04888839983AA83BB83BC01CD0187
:104A70009F77DF91CF91FF90EF90DF90CF90BF9025
:104A8000AF909F908F9008950E94F924089584E23A
:104A900091E00E94F9240895609324017093250108
:104AA0008093260190932701089597F99F6780E8E6
:104AB00070E060E008959FEF80EC089500240A9470
:104AC0001616170618060906089500240A941216E9
:104AD0001306140605060895092E0394000C11F41C
:104AE000882352F0BB0F40F4BF2B11F460FF04C0C9
:104AF0006F5F7F4F8F4F9F4F089557FD9058440F22
:104B0000551F59F05F3F71F04795880F97FB991F2C
:104B100061F09F3F79F087950895121613061406E9
:104B2000551FF2CF4695F1DF08C016161706180676
:104B3000991FF1CF86957105610508940895E89451
:104B4000BB2766277727CB0197F90895052E97FB9A
:104B50001EF400940E94BD2557FD07D00E940F2629
:104B600007FC03D04EF40C94BD255095409530952C
:104B700021953F4F4F4F5F4F0895909580957095C9
:104B800061957F4F8F4F9F4F08950E943126A59FBB
:104B9000900DB49F900DA49F800D911D1124089538
:104BA000B7FF0C94C5250E94C525821B930B089561
:104BB0002F923F924F925F926F927F928F929F922D
:104BC000AF92BF92CF92DF92EF92FF920F931F931B
:104BD000CF93DF93CDB7DEB7CA1BDB0B0FB6F894CC
:104BE000DEBF0FBECDBF09942A88398848885F840C
:104BF0006E847D848C849B84AA84B984C884DF807D
:104C0000EE80FD800C811B81AA81B981CE0FD11D60
:104C10000FB6F894DEBF0FBECDBFED010895A1E23F
:104C20001A2EAA1BBB1BFD010DC0AA1FBB1FEE1F26
:104C3000FF1FA217B307E407F50720F0A21BB30B71
:104C4000E40BF50B661F771F881F991F1A9469F7ED
:104C500060957095809590959B01AC01BD01CF0149
:104C60000895A29FB001B39FC001A39F700D811D45
:104C70001124911DB29F700D811D1124911D089565
:104C80000E9454260C946C250E94652558F00E94C1
:104C90005E2540F029F45F3F29F00C945525511111
:104CA0000C94A0250C945B250E947D2568F3992324
:104CB000B1F3552391F3951B550BBB27AA27621718
:104CC0007307840738F09F5F5F4F220F331F441F25
:104CD000AA1FA9F335D00E2E3AF0E0E832D0915059
:104CE0005040E695001CCAF72BD0FE2F29D0660F46
:104CF000771F881FBB1F261737074807AB07B0E889
:104D000009F0BB0B802DBF01FF2793585F4F3AF08E
:104D10009E3F510578F00C9455250C94A0255F3FDB
:104D2000E4F3983ED4F3869577956795B795F79514
:104D30009F5FC9F7880F911D9695879597F90895FC
:104D4000E1E0660F771F881FBB1F62177307840798
:104D5000BA0720F0621B730B840BBA0BEE1F88F7A7
:104D6000E09508950E94B9266894B1110C94A0258D
:104D700008950E94852588F09F5798F0B92F9927AC
:104D8000B751B0F0E1F0660F771F881F991F1AF036
:104D9000BA95C9F714C0B13091F00E949F25B1E0D7
:104DA00008950C949F25672F782F8827B85F39F0D6
:104DB000B93FCCF3869577956795B395D9F73EF4CF
:104DC00090958095709561957F4F8F4F9F4F089577
:104DD000DB018F939F930E94C525BF91AF91A29F46
:104DE000800D911DA39F900DB29F900D11240895E9
:104DF000991B79E004C0991F961708F0961B881F2D
:104E00007A95C9F780950895AA1BBB1B51E107C08D
:104E1000AA1FBB1FA617B70710F0A61BB70B881F4A
:104E2000991F5A95A9F780959095BC01CD010895D9
:104E300097FB072E16F4009407D077FD09D00E9447
:104E4000042707FC05D03EF4909581959F4F089567
:104E5000709561957F4F0895EE0FFF1F0590F491B7
:104E6000E02D09940E943126B7FF0895821B930B11
:104E7000089597FB57FF0C9449279F938F930E94A7
:104E800049276E1B7F0BAF91BF918A0B9B0B089537
:104E9000E894DF93CF93FC01DB010E9431267F93DE
:104EA0006F93E9019A01AC01BF93AF933F932F93A6
:104EB000DF010E94312626F46C1B7D0B820B930BC5
:104EC0009E01EB01FC010E941328AF91BF912F912D
:104ED0003F910E941328BE01CF01F9012F913F910C
:104EE000CF91DF910895689401C0E894F92FF12BD8
:104EF00012F00C94A727A0E0B0E0E1E8F7E20C94F0
:104F0000DE25092E059422F40E940328112392F431
:104F1000F0E80F26FFEFE094F09400951095B09420
:104F2000C094D094A194BF0ACF0ADF0AEF0AFF0A07
:104F30000F0B1F0B0E94B22707FC0E940328CDB75E
:104F4000DEB7ECE00C94FA25689401C0E8948F92E7
:104F50009F92CF93DF930E94B227DF91CF919F90D2
:104F60008F90089588249924F401E401B0E49F937C
:104F7000AA279A158B049C04ED05FE05CF05D007E2
:104F8000A10798F4AD2FDC2FCF2FFE2FE92D982C01
:104F9000892E982F872F762F652F542F432F322F4E
:104FA0002227B85031F7BF9127C01B2EBF91BB27D6
:104FB000220F331F441F551F661F771F881F991F1D
:104FC000881C991CEE1FFF1FCC1FDD1FAA1FBB1FD3
:104FD0008A149B04EC05FD05CE05DF05A007B1078B
:104FE00048F08A189B08EC09FD09CE09DF09A00BDF
:104FF000B10B21601A94E1F62EF49401AF01BE01C9
:10500000CD01000C08956095709580959095309530
:105010004095509521953F4F4F4F5F4F6F4F7F4FBA
:105020008F4F9F4F08950E943126460F571FC81F6C
:10503000D91F08F4319608950F931F93CF93DF93F0
:10504000869F8001879F100D969F100D1124C80127
:105050000E943828EC01009729F0A80160E070E078
:105060000E943D2ACE01DF91CF911F910F910895AB
:10507000CF93DF938230910510F482E090E0E091CD
:10508000E504F091E60420E030E0C0E0D0E03097A5
:1050900011F14081518148175907C0F0481759074D
:1050A00061F482819381209719F09B838A832BC0BE
:1050B0009093E6048093E50426C02115310519F08C
:1050C0004217530718F49A01BE01DF01EF01028075
:1050D000F381E02DDCCF2115310509F1281B390BB7
:1050E0002430310590F412968D919C91139761159F
:1050F000710521F0FB019383828304C09093E60441
:105100008093E504FD01329644C0FD01E20FF31FD8
:1051100081939193225031092D933C933AC0209171
:10512000E3043091E404232B41F420912A013091CF
:105130002B013093E4042093E30420912801309163
:1051400029012115310541F42DB73EB740912C01BD
:1051500050912D01241B350BE091E304F091E40400
:10516000E217F307A0F42E1B3F0B2817390778F03E
:10517000AC014E5F5F4F2417350748F04E0F5F1F9D
:105180005093E4044093E3048193919302C0E0E0E0
:10519000F0E0CF01DF91CF9108950F931F93CF934C
:1051A000DF93009709F48CC0FC01329713821282BE
:1051B0000091E5041091E6040115110581F42081A8
:1051C0003181820F931F2091E3043091E40428176A
:1051D000390779F5F093E404E093E30471C0D80152
:1051E00040E050E0AE17BF0750F412962D913C916D
:1051F0001397AD012115310509F1D901F3CF9D01B7
:10520000DA013383228360817181860F971F8217B1
:10521000930769F4EC0128813981260F371F2E5F2F
:105220003F4F318320838A819B8193838283452BE7
:1052300029F4F093E604E093E50442C01396FC934E
:10524000EE931297ED01499159919E01240F351F5C
:10525000E217F30771F480819181840F951F029604
:1052600011969C938E938281938113969C938E9337
:105270001297E0E0F0E0D80112968D919C9113977F
:10528000009719F0F8018C01F6CF8D919C9198014F
:105290002E5F3F4F820F931F2091E3043091E4046F
:1052A0002817390769F4309729F41092E604109210
:1052B000E50402C0138212821093E4040093E30415
:1052C000DF91CF911F910F910895A0E0B0E0EBE640
:1052D000F9E20C94DC25EC01009721F4CB010E944B
:1052E0003828B8C0FC01E60FF71F9C012250310995
:1052F000E217F30708F4ACC0D9010D911C91119786
:1053000006171707B0F00530110508F49FC0C80153
:1053100004978617970708F499C002501109061BD5
:10532000170B019311936D937C93CF010E94CD28AD
:105330008DC05B01A01AB10A4C01800E911EA09194
:10534000E504B091E60440E050E0E12CF12C109728
:1053500009F44AC0A815B905D1F56D907C90119754
:10536000630182E0C80ED11CCA14DB0480F1A301E2
:105370004A195B096A0182E0C80ED11C1296BC90E2
:1053800012971396AC91B5E0CB16D10440F0B282DF
:10539000A38351834083D9016D937C930AC00E5F30
:1053A0001F4FC301800F911FF90191838083EB2D63
:1053B000FA2FE114F10431F0D7011396FC93EE9328
:1053C000129744C0F093E604E093E5043FC08D914A
:1053D0009C9111974817590708F4AC017D0112966A
:1053E0000D90BC91A02DB3CF8091E3049091E40483
:1053F00088159905E1F446175707C8F480912801EC
:1054000090912901009741F48DB79EB740912C01EE
:1054100050912D01841B950BE817F907C8F4F09300
:10542000E404E093E304F901718360830FC0CB01CE
:105430000E9438287C01009759F0A801BE010E9403
:10544000342ACE010E94CD28C70104C0CE0102C07B
:1054500080E090E0CDB7DEB7EEE00C94F82581E077
:1054600090E0F8940C94442AFB01DC0102C0019006
:105470000D9241505040D8F70895DC0101C06D9362
:1054800041505040E0F7089510E0C4EED0E004C071
:10549000FE010E942C272196C53ED107C9F7F8943A
:0254A000FFCF3C
:1054A2000F00F401D00704000401340C340C340C56
:1054B200340C340C0000803FFFFFFFFF00E10000CE
:1054C20000000000010000000000E704800004006A
:1054D2000F0020003700550078009C01B501CF0174
:1054E200EA0107022602470269028E02B502DE02C3
:1054F2000A03018001800180FF7FFF7FFF7F0000A0
:1055020000004417B116DC168B170D17EB16FF16A9
:1055120000000000BC0BE70D7F0CD20BDD0BA70CCB
:10552200830C00000000B6028602E6025A027E02E6
:105532006A025B02000000005A0D000000006C0EBF
:1055420000000000C612000000006C0E00C1808145
:10555200000000426C7565746F6F746876657262E4
:10556200696E64756E672068657267657374656CD1
:105572006C74004665686C65722044726568626589
:10558200776567756E677373656E736F72730046C6
:1055920065686C65722042657363686C65756E69D7
:1055A20067756E677373656E736F7273000D0A00B1
:00000001FF
